:020000040000FA
:100000000000000033288207000016341534123433
:10001000113410340134A0001620A00B0C28080065
:10002000A10064300B20A10B11280800C63000008D
:10003000FF3E031D172800000000000008003030BC
:10004000A200A301A30A2308073C031921282308BF
:100050000320850022080B20A20AA20A2208803C65
:10006000031D2228080083120730990009308B00F5
:100070008316FF2390009F01E830850081139516B9
:100080009616831220300B2005080B108316FF30C4
:10009000850063000000E8308500831205080B101E
:1000A00005300B2017308500A401A40A2408073A64
:1000B000031D5D28A401A40A6028000000000000C0
:1000C000851E55281F20240803208500D030A50058
:1000D00001301020851E5228A50B6828FE30A5008F
:1000E00024080320850025087C2017308500250979
:1000F0007C20A50B70284428A000851E52281630AD
:10010000A100A10B8128A00B7D28080020344534D4
:100110006C3465346334743472346F346E346934DF
:1001200063342034443469346534203466346F34A5
:100130007234203431343234463436343734353442
:1001400020342D34203450346534743465342034F4
:1001500047347234693466346634693474346834CC
:100160007334203432343034303434342E34203448
:10017000523436342E34313437343034353432342A
:0601800030343034343449
:02400E00843FED
:00000001FF
